:100000000C943A000C9457000C9457000C94570031
:100010000C9457000C9457000C9457000C94570004
:100020000C9457000C9457000C9457000C945700F4
:100030000C9457000C9457000C9457000C945700E4
:100040000C9457000C9457000C9457000C945700D4
:100050000C9457000C9457000C9457000C945700C4
:100060000C9457000C9457000C9457000C945700B4
:100070000C94570011241FBECFEFD2E0DEBFCDBFDE
:1000800011E0A0E0B1E0E4E8FEE002C005900D92CE
:10009000A031B107D9F711E0A0E1B1E001C01D9294
:1000A000A831B107E1F70E9459000C9441070C9464
:1000B0000000EF92FF920F931F93CF93DF93CDB782
:1000C000DEB7A7E2B0E0E7E2F0E0808180648C93E5
:1000D000A1E8B0E0E1E8F0E08081982F88EF892383
:1000E00081608C93A0E8B0E0E0E8F0E090818CEFD4
:1000F00089238C93A1E8B0E0E1E8F0E08081982FBB
:1001000098608FEE89238C93809104019091050172
:10011000A0910601B09107018E339105A105B105AB
:100120000CF054C0E1E6F0E080E88083E1E6F0E026
:1001300083E080838091000190910101A0910201F0
:10014000B091030128E030E040E050E0BC01CD0177
:100150000E94CD06DA01C90180930001909301014C
:10016000A0930201B09303018091040190910501D5
:10017000A0910601B091070188309105A105B10554
:1001800064F5A1E8B0E0E1E8F0E08081982F88EF25
:10019000892382608C938091000190910101A0914C
:1001A0000201B091030128E030E040E050E0BC01E2
:1001B000CD010E94CD06DA01C90180930001909320
:1001C0000101A0930201B093030107C0E1E6F0E052
:1001D00080E88083E1E6F0E0108280910001909158
:1001E0000101A0910201B0910301BC01CD010E9467
:1001F0003A047B018C018091040190910501A0914A
:100200000601B0910701BC01CD010E943A04DC0156
:10021000CB019C01AD01C801B7010E944A03DC017A
:10022000CB0120E030E040E85FE3BC01CD010E945B
:10023000EC02DC01CB018093100190931101A0939B
:100240001201B09313018091000190910101A091DE
:100250000201B09103012091040130910501409108
:10026000060150910701BC01CD010E94CD06DA01C3
:10027000C9010197A109B109809314019093150157
:10028000A0931601B0931701E0901001F0901101B6
:1002900000911201109113018091140190911501A8
:1002A000A0911601B0911701BC01CD010E943A0442
:1002B000DC01CB019C01AD01C801B7010E94EC0239
:1002C000DC01CB0120E030E040E05FE3BC01CD0188
:1002D0000E941D03DC01CB0180931001909311015A
:1002E000A0931201B093130180911001909111011C
:1002F000A0911201B091130120E030E040E85FE3EB
:10030000BC01CD010E94040488230CF413C0809129
:10031000140190911501A0911601B0911701019659
:10032000A11DB11D8093140190931501A093160196
:10033000B0931701A0E8B0E0E0E8F0E080818F77AB
:1003400080648C93E9E8F0E08091140190911501AC
:10035000A0911601B0911701892F9A2FAB2FBB27BF
:10036000A7FDBA958083E8E8F0E0809114019091B0
:100370001501A0911601B09117018083FFCFA0E075
:10038000B0E0E5ECF1E00C940E07FC016A0190810D
:10039000923008F41BC1DB018C91823080F09430E4
:1003A00061F4843009F012C19181EB0189819817C1
:1003B00009F40CC1E8E0F1E009C1843011F4FB015B
:1003C00005C1823091F4923009F000C1EA01DF01E9
:1003D00088E00D9009928150E1F78181FB019181C4
:1003E0008923E6018983F601F1C0923041F36280EE
:1003F0007380EB018A809B80E480F5800681178101
:100400002C813D814E815F815301A818B908C50137
:10041000B7FCABC080970CF457C0861497040CF45B
:10042000BEC03401EE24FF2487019181FB0181814C
:10043000981709F4A6C0992309F49CC02E193F0906
:10044000400B510B57FDB0C0E60119827B826A82D6
:10045000F6012483358346835783E6012C813D8151
:100460004E815F8179018A01DA01C9010197A109F1
:10047000B1098F5F9F4FAF4FBF43F8F4E6016A8128
:100480007B81A8019701220F331F441F551F615024
:10049000704079018A01DA01C9010197A109B10906
:1004A0008F5F9F4FAF4FBF4360F3E6017B836A834B
:1004B000F601248335834683578383E0D6018C93EA
:1004C00057FD39C0F60182C086149704B4F4C0E029
:1004D000D0E0DA01C90181709070A070B0705695BB
:1004E000479537952795282B392B4A2B5B2B21963F
:1004F000AC16BD0671F78A0C9B1C681479040CF0CD
:1005000094CFC0E0D0E05401A618B708D801C701C5
:1005100081709070A070B07016950795F794E7946D
:10052000E82AF92A0A2B1B2B2196AC16BD0671F777
:100530006A0C7B1C7ACFDA01C901B695A79597950D
:1005400087952170307040705070282B392B4A2BC2
:100550005B2BE6012C833D834E835F838A819B81E5
:1005600001969B838A83F60131C0882799278A19CF
:100570009B0950CFE21AF30A040B150BA80197014F
:1005800061CFE60199837B826A822E0D3F1D401F59
:10059000511FF60124833583468357838ECF20E095
:1005A00030E040E050E041CF81E0E60189837B828A
:1005B0006A8250954095309521953F4F4F4F5F4F40
:1005C000F601248335834683578347CFCF01EEE07E
:1005D000CDB7DEB70C942A07A0E2B0E0E2EFF2E07C
:1005E0000C94160769837A838B839C832D833E83C7
:1005F0004F83588789E1E82EF12CEC0EFD1EB701E0
:10060000CE0101960E94C5058E010F5E1F4FB801F5
:10061000CE0105960E94C5058A8991E089278A8BBB
:10062000AE01475F5F4FB801C7010E94BF010E9442
:10063000A304E6E0A0960C943207A0E2B0E0E3E267
:10064000F3E00C94160769837A838B839C832D8354
:100650003E834F83588799E1E92EF12CEC0EFD1E65
:10066000B701CE0101960E94C5058E010F5E1F4F96
:10067000B801CE0105960E94C505AE01475F5F4FE8
:10068000B801C7010E94BF010E94A304E6E0A09642
:100690000C943207A8E1B0E0E0E5F3E00C94100719
:1006A00069837A838B839C832D833E834F83588712
:1006B000B1E18B2E912C8C0E9D1EB401CE010196C2
:1006C0000E94C5058E01075F1F4FB801CE01059638
:1006D0000E94C5052989223008F46AC03985323064
:1006E00008F468C08A899A8589278A8B243009F49E
:1006F00063C0223009F460C0343041F41D8A1E8A80
:100700001F8A188E1C8A1B8AB40177C0323009F404
:1007100058C06B897C898B859C85681B790B7C8B89
:100720006B8B2D893E894F89588DED84FE840F8512
:1007300018892E153F054007510740F4220F331F3B
:10074000441F551F615070407C8B6B8B80E090E0A4
:10075000A0E0B0E4AA24BB24650160E070E02E159F
:100760003F054007510740F0A82AB92ACA2ADB2AC8
:100770002E193F09400B510BB695A7959795879574
:10078000220F331F441F551F6F5F7F4F6F3171055D
:1007900031F7D601C5018F779070A070B0708034AA
:1007A0009105A105B10589F0AD8ABE8ACF8AD88EA0
:1007B000B40123C0B80121C03217D1F768E071E05D
:1007C0001CC084E0898BB40118C0A7FCEDCF2115B3
:1007D00031054105510541F380E490E0A0E0B0E02F
:1007E000A80EB91ECA1EDB1E80E89FEFAFEFBFEF59
:1007F000A822B922CA22DB22D7CFCB010E94A304B0
:10080000ECE068960C942C07A8E1B0E0EAE0F4E094
:100810000C94160769837A838B839C832D833E8394
:100820004F83588781E1E82EF12CEC0EFD1EB701B5
:10083000CE0101960E94C5058E01075F1F4FB801CA
:10084000CE0105960E94C5058989823018F42FEFE4
:100850003FEF0BC089858230D0F3B801C7010E94F9
:100860006406282F332727FD3095C901E6E06896F6
:100870000C943207A8E0B0E0E0E4F4E00C9419072F
:100880009B01AC0183E089831A8257FD51C0211579
:1008900031054105510539F482E08983CE01019685
:1008A0000E94A3044CC0EEE1F0E0FC83EB838A815C
:1008B0008823C9F1203010E0310710E0410710E82B
:1008C0005107C9F188279927DC01821B930BA40BE0
:1008D000B50B8D839E83AF83B8872D813E814F8179
:1008E0005885203080E0380780E0480780E45807CA
:1008F000A8F6EB81FC81DA01C901880F991FAA1FB4
:10090000BB1F31979C01AD01803010E0910710E0D2
:10091000A10710E4B10778F3FC83EB838D839E83FA
:10092000AF83B887BBCF2D833E834F835887D5CF06
:1009300081E08A83ACCF60E070E080E09FECE3E090
:1009400028960C9435074F925F926F927F928F9208
:100950009F92AF92BF92DF92EF92FF920F931F93FD
:1009600020E030E040E050E0FC01E480F5800681CA
:100970001781D1808081823038F4D801C701A0610D
:10098000AF77B0706FEFD9C0843009F46EC0823099
:1009900009F471C0E114F1040105110509F46BC0FB
:1009A000828193816FEF823896070CF06AC062E80B
:1009B0007FEF681B790B6A3171050CF080C047012D
:1009C0005801062E04C0B694A794979487940A946D
:1009D000D2F744245524320181E090E0A0E0B0E059
:1009E00004C0880F991FAA1FBB1F6A95D2F70197F1
:1009F000A109B109E822F9220A231B23E114F10419
:100A00000105110529F061E0462E512C612C712C55
:100A100085017401E428F52806291729D801C701A2
:100A20008F779070A070B07080349105A105B105EA
:100A300009F457C0D801C701CF96A11DB11D60E0D0
:100A400070E08030E0E09E07E0E0AE07E0E4BE0743
:100A500010F061E070E027E0B695A795979587952F
:100A60002A95D1F7AF77B07068C080E090E0A0E041
:100A7000B0E06FEF62C080E090E0A0E0B0E060E046
:100A80005CC0803891058CF7BC0161587F4FD8015C
:100A9000C7018F779070A070B07080349105A10568
:100AA000B105A1F08FE390E0A0E0B0E0E80EF91E00
:100AB0000A1F1B1F17FD28C0D801C701CCCF60E05B
:100AC00070E080E090E0A0E0B0E0CCCFE7FEF2CFB5
:100AD00080E490E0A0E0B0E0E80EF91E0A1F1B1FC2
:100AE000E9CFE7FC18C080E090E060E0E61660E047
:100AF000F60660E0060760E4160710F081E090E07B
:100B0000BC01D801C701A7CF16950795F794E794C4
:100B10006F5F7F4FD1CFD801C701805C9F4FAF4F30
:100B2000BF4F60E070E08030E0E09E07E0E0AE079D
:100B3000E0E4BE0708F48FCF8CCF282F392F9A2FEF
:100B40009F77842F8078892B962F97959927979553
:100B50008F77482F492B6695852F8078862BD794E1
:100B6000DD24D7948F77582F5D29CA01B9011F91D1
:100B70000F91FF90EF90DF90BF90AF909F908F907C
:100B80007F906F905F904F900895FC01DB01208172
:100B900031819281492F4F7750E0991F9927991FF2
:100BA0008381682F660F692B881F8827881FFD01A6
:100BB0008183662309F049C021153105410551059E
:100BC00009F470C082E89FEFFD0193838283220FB6
:100BD000331F441F551F220F331F441F551F220F61
:100BE000331F441F551F220F331F441F551F220F51
:100BF000331F441F551F220F331F441F551F220F41
:100C0000331F441F551F83E08C932030F0E03F07D3
:100C1000F0E04F07F0E45F0790F482E89FEF220FC7
:100C2000331F441F551F0197203060E0360760E0F6
:100C3000460760E4560798F3FD0193838283FD0124
:100C4000248335834683578308956F3F71F1862F40
:100C500099278F579040FD019383828383E08C9383
:100C6000220F331F441F551F220F331F441F551FD0
:100C7000220F331F441F551F220F331F441F551FC0
:100C8000220F331F441F551F220F331F441F551FB0
:100C9000220F331F441F551F50642483358346831E
:100CA0005783089582E08C930895211531054105FD
:100CB000510519F484E08C93089544FD02C01C9200
:100CC000BECF81E08C93BBCFEF92FF920F931F9327
:100CD000CF93DF93FC01DB018081823050F09C9147
:100CE000923038F0843041F49430B1F0818188231F
:100CF00081F461E070E04BC09430E9F18230A1F002
:100D00009230A1F36181ED018981681791F066232A
:100D100081F36FEF7FEF3BC0EB018981682F77276D
:100D20008181681B710933C0923059F560E070E031
:100D30002EC022813381ED018A819B818217930726
:100D400034F3281739079CF0E480F5800681178179
:100D5000FD0124813581468157812E153F054007CD
:100D60005107A8F2E216F30604071507F8F6662302
:100D700009F0BFCFCECFFB018181882309F0B9CF25
:100D8000C8CFEB018981882309F0B3CFC2CFCB0153
:100D9000E6E0CDB7DEB70C94320797FB092E0526A7
:100DA0000ED057FD04D014D00AD0001C38F4509552
:100DB0004095309521953F4F4F4F5F4F0895F6F77F
:100DC00090958095709561957F4F8F4F9F4F0895B7
:100DD000A1E21A2EAA1BBB1BFD010DC0AA1FBB1F3F
:100DE000EE1FFF1FA217B307E407F50720F0A21BB1
:100DF000B30BE40BF50B661F771F881F991F1A941E
:100E000069F760957095809590959B01AC01BD0147
:100E1000CF0108952F923F924F925F926F927F92EF
:100E20008F929F92AF92BF92CF92DF92EF92FF92FA
:100E30000F931F93CF93DF93CDB7DEB7CA1BDB0BA6
:100E40000FB6F894DEBF0FBECDBF09942A8839884B
:100E500048885F846E847D848C849B84AA84B98452
:100E6000C884DF80EE80FD800C811B81AA81B9815E
:100E7000CE0FD11D0FB6F894DEBF0FBECDBFED0172
:040E80000895FFCF03
:100E8400A0093D00762701000000000000000000DA
:00000001FF
